:0200000480007A
:10000000ADA8010001000100010001000100010094
:10001000232E11FE232C51FE232A61FE232871FE7C
:100020002326A1FE2324B1FE2322C1FE2320D1FEDC
:10003000232EE1FC232CF1FC232A01FD232811FDB2
:100040002326C1FD2324D1FD2322E1FD2320F1FD40
:100050003971AD28F250E2525253C2533255A25573
:10006000125682567247E2475248C248324EA24E5A
:10007000124F824F2161730020309741000093811D
:10008000E182176100001301E1041385C1819765C6
:1000900000009385E5C36306B50023200500110524
:1000A000DDBF1735000013052500711197350000DD
:1000B000938585FF6308B500144111052AC0829617
:0C00C0000245EDB71101EF20F00001A097
:1000CC00828003C75183930710046303F700828077
:1000DC001C4103A7C183A507998F1CC1828003A66D
:1000EC00418409C6184218C103A6418483A5C18363
:1000FC00310629456F00806C41114AC083A74184A9
:10010C0022C40041984326C283AE470003AE870049
:10011C0003A3070183A8470103A887018C53D0537D
:10012C00945706C6AA84C84FDC5718C0984048CCD0
:10013C005CD42322D40195472324C40123286400D2
:10014C00232A1401232C04010CD050D014D4DCC469
:10015C005CC418C0228561375C40B1CF9C40B24072
:10016C00224483AF070003AF470083AE870003AE82
:10017C00C70003A3070183A8470103A88701CC4F3D
:10018C009053D4539857DC5723A0F40123A2E401D5
:10019C0023A4D40123A6C40123A8640023AA140118
:1001AC0023AC0401CCCC90D0D4D098D4DCD402496C
:1001BC0092444101828088449947930584005CC431
:1001CC00EF00E06983A7418448441306C4009C43B4
:1001DC00B24092441CC022440249A94541016F001F
:1001EC00E05D83C7518383A681839387F7FB93B725
:1001FC001700D58F23ACF18213072004238AE182E8
:10020C00828013071004A38AE18223AC01828280CE
:10021C0035711305000306CF22CDE6DAEED626CBD8
:10022C004AC94EC752C556C35AC1DEDEE2DCEAD813
:10023C00EF00407123A0A18413050003EF00807030
:10024C0083A7018423A2A1841CC189471CC5B7358F
:10025C000080930780025CC57D469385C58E232262
:10026C0005004105EF00407E37370080930747E5D6
:10027C00032E47E503A3470083A8870003A8C70004
:10028C008C4BD04B944F03D7C70183C7E701B73DC5
:10029C000080231EE102230FF1021387CD1BA94717
:1002AC002945232EF76472D01AD246D442D62ED8C2
:1002BC0032DA36DCEF00E077373500801305C59075
:1002CC00EF00C0742945EF00C07683A70183638ECD
:1002DC00074A373500801305C593EF002073294575
:1002EC00EF0020753735008013058599EF00A06766
:1002FC002945EF000074373500809305800C1305F9
:10030C00059DEF004066EF00607337340080832753
:10031C0044E7373D0080032C4DE93EC623A6A1825D
:10032C008549130444E78944E93D653D8347E4016D
:10033C005048032E4400032384008328C400032860
:10034C000401144C0357C401B24E230FF1048C006A
:10035C0085470810B2CA3ECE26CAF6C0F2C29AC46D
:10036C00C6C6C2C8B6CC231EE10455295246133565
:10037C00150023ACA18263C0C40293172600B29768
:10038C00F51732858D4530083ECC0D2952460506B1
:10039C0032CAE3D4C4FEE2461385C1849385CD1BD7
:1003AC00152103A54184930A10040D4AB13303C7E8
:1003BC00418393070004130B4DE963F1E702568563
:1003CC00930530048921F24713871A006306F5362A
:1003DC0083C74183937AF70FE3F357FFD247624BFE
:1003EC004808330AFA028509B34A6A0356CAD13956
:1003FC009307900CE39AF9F2EF00406423A4A182D6
:10040C0037350080130505A0EF0040602945EF004B
:10041C00406237350080130505A1EF00205F2945A8
:10042C00EF00206183A5C18337350080130585A4B7
:10043C00373400800D2B9545130544A62D2383A539
:10044C00818337350080130505A8312B85451305AD
:10045C0044A6112B83C55183373500801305C5A9DC
:10046C001923B734008093051004138584ABE52958
:10047C0083C5418337350080130545ADED219305C8
:10048C002004138584ABC5219387C1848C533735E5
:10049C000080130505AFC1299D45130544A6E12134
:1004AC00B73700809387C71B83A5C7653735008096
:1004BC001305C5B04D2937350080130585B2EF0003
:1004CC00E05437350080130545B5EF00205403A7E1
:1004DC004184B7370080138507B60C433EC6373DC1
:1004EC0000805121373500801305C5B7052303A7BC
:1004FC0041841305CDBA373C00804C43B73B008098
:10050C00B73900808D218145130544A6A92903A77D
:10051C00418413058CBC373900800C47330A6A417F
:10052C0099218945130544A63D2903A741841385C8
:10053C004BBE4C470D29C545130544A62D2183A55B
:10054C004184138509C0C10539291305C9C17D2909
:10055C0037350080130505C5552903A70184B2471B
:10056C000C43138507B6012137350080130505C6EA
:10057C00712983A701841305CDBACC43ED2681459F
:10058C00130544A6CD2683A7018413058CBC8C4788
:10059C00D92E8545130544A6F92683A70184138516
:1005AC004BBECC47C926C945130544A66D2E83A561
:1005BC000184138509C0C1057D261305C9C1B92164
:1005CC00D24537350080130505CA712E95451305A4
:1005DC0044A6512E93173A00338A47413735008091
:1005EC00B3055A411305C5CBBD2EB545130544A61D
:1005FC009D2EE24537350080130585CDAD269D45F2
:10060C00130544A68D26F24537350080130545CFDA
:10061C00992E8545130544A6B926373500800C1054
:10062C00130505D18926373500801305C5D2F92E5F
:10063C00373500808C00130505D6352637350080FC
:10064C001305C5D7E1262945ED2603A7C18283A54D
:10065C0081829307301F998D23A2B18263DFB71279
:10066C0037350080130585E0FD2C03A54182EF1082
:10067C0070642A84EF105076B737008003A6870A7F
:10068C0083A6C70AEF009050B737008003A6070B6C
:10069C0083A6470BEF008061EF20C00423A0A1824A
:1006AC00B737008003A5870BA285EF10E02B23AE94
:1006BC00A180373500801305C5E1752403A541825F
:1006CC00EF10505FB7370080AA8503A5C70BEF105A
:1006DC00A0292A84EF101057AA84EF10B05DAA85C8
:1006EC002285EF10B00EB737008083A5070CEF10F2
:1006FC00A05BEF1030552A8437350080A685130592
:10070C00C5E49524A54763D7870A37350080A285B1
:10071C00130505E5892C2945292EFA406A44DA444B
:10072C004A49BA492A4A9A4A0A4BF65B665CD65C35
:10073C00465DB65D0D6182806C0801450D22032378
:10074C004B0083288B000328CB0003250B0183254A
:10075C004B0103268B018356CB010347EB0183C767
:10076C004183850AE2C09AC2C6C4C2C6AAC8AECA30
:10077C00B2CC231ED104230FE10423AE318393FAB0
:10078C00FA0F4E8AE3FD57C391B937350080130534
:10079C008596AD2C2945712CB1B6373500801305E3
:1007AC0005DBAD2437350080130585DE852429450E
:1007BC004924A5B713050003AD2C81BF0905AA95E3
:1007CC000CC28280130756001308800C33080703F1
:1007DC000A06931727003E9514C138DD54C1B307A0
:1007EC00C800AE97944BD8CB98CF1387160098CBF4
:1007FC001C41C295B2950566B29523AAF5FA154728
:10080C0023AEE18282801375F50F93F5F50F630427
:10081C00B50001458280A38AA182054582804111E1
:10082C0022C426C206C62A84AE8483C5340003457E
:10083C002400D13F7DF9A6852285DD2C81476356A6
:10084C00A000294723AEE1828547B240224492445E
:10085C003E85410182807915133515008280411146
:10086C0022C426C206C62A84AE84F53715C180C0C0
:10087C0085476304F40205C80947630DE4029147F8
:10088C006313F40098C0B240224492444101828028
:10089C008D479CC08547E310F4FE03A7C1839307E3
:1008AC00400663DFE700B240224423A004009244D8
:1008BC0041018280B24022449CC09244410182801A
:1008CC00B24022448D479CC0924441018280411128
:1008DC0022C406C62A840345050011C50504912AC5
:1008EC000345040065FDB24022444101828091A27F
:1008FC00797126D206D622D44AD0AA84634E050238
:10090C000A894A84294799E0631C2401B3E7E4026D
:10091C00050493870703B3C4E402A30FF4FEE5B701
:10092C007D1403450400E137E31C24FFB25022542C
:10093C0092540259456182801305D0024D3FB30495
:10094C0090407DBF03A78184B307A7003765008063
:10095C0023A4F1841305C58C930600403A9563D308
:10096C00F600029082805D7152CC06D622D426D23B
:10097C004AD04ECE56CA2A8A03450500BEC25C1820
:10098C002EDA32DC36DEBAC0C2C4C6C63EC61DC1C3
:10099C000144930A5002930430061309300793095B
:1009AC00400663025503A1370504B3078A0003C54B
:1009BC00070065F9B250225492540259F249624A26
:1009CC00D24A61618280930614003307DA0031A0A9
:1009DC0063822703638637038506834707003684C3
:1009EC000507F9D3E39697FEB247884391073EC6B5
:1009FC00FD3D5DBFB247884391073EC6C93D6DB70B
:100A0C00B247884391073EC6E53579BF411122C4F0
:100A1C0006C62A840345050011C50504192803459B
:100A2C00040065FD29453120B240224401454101B5
:100A3C008280B70710F023A0A7F08280B70710F0D0
:100A4C0003A507F182800000B3C7A50093F7370018
:100A5C003307C500639607009307300063E4C702B1
:100A6C0093070500636CE5006780000083C60500F2
:100A7C009387170093851500A38FD7FEE3E8E7FE55
:100A8C006780000093773500639207089307050091
:100A9C009376C7FF138606FE63F6C70883A305008B
:100AAC0083A2450083AF850003AFC50083AE05016B
:100ABC0003AE450103A3850183A8C50193854502B7
:100ACC009387470203A8C5FF23AE77FC23A057FEEC
:100ADC0023A2F7FF23A4E7FF23A6D7FF23A8C7FF72
:100AEC0023AA67FE23AC17FF23AE07FF6FF0DFFAD4
:100AFC0083C605009387170093851500A38FD7FE37
:100B0C0093F63700E39606FE6FF09FF89307050007
:100B1C006FF01FFF03A605009387470093854500E0
:100B2C0023AEC7FEE3E8D7FEE3EAE7F467800000F4
:100B3C003367B5009303F0FF13773700631007108A
:100B4C00B7877F7F9387F7F70326050083A60500F9
:100B5C00B372F6003363F600B382F200B3E26200C4
:100B6C00639272106316D6080326450083A64500CF
:100B7C00B372F6003363F600B382F200B3E26200A4
:100B8C00639E720C6316D6060326850083A6850029
:100B9C00B372F6003363F600B382F200B3E2620084
:100BAC006398720C6316D6040326C50083A6C50091
:100BBC00B372F6003363F600B382F200B3E2620064
:100BCC006392720C6316D6020326050183A60501F7
:100BDC00B372F6003363F600B382F200B3E2620044
:100BEC00639C720A1305450193854501E30ED6F407
:100BFC001317060193970601631EF700135706019E
:100C0C0093D706013305F7409375F50F63900502F2
:100C1C00678000001357070193D707013305F7408E
:100C2C009375F50F63940500678000001377F70F39
:100C3C0093F7F70F3305F740678000000346050074
:100C4C0083C6050013051500938515006314D600A3
:100C5C00E31606FE3305D6406780000013054500F9
:100C6C0093854500E31CD6FC13050000678000004B
:100C7C001305850093858500E312D6FC130500004F
:100C8C00678000001305C5009385C500E318D6FAEC
:100C9C00130500006780000013050501938505010D
:100CAC00E31ED6F81305000067800000130101FD58
:100CBC0023248102232291022328610113040500BD
:100CCC00130B0500B704100013D545012320210395
:100CDC00232E3101232671019384F4FF2326110264
:100CEC00232C4101232A51011375F57F930B060028
:100CFC0093890600B3F4B40013D9F5016306050A11
:100D0C009307F07F6306F51093943400B7068000C8
:100D1C00B3E4D400935ADB01B3EA9A0013143B00FA
:100D2C00130A15C0130B000013D54901B7041000AA
:100D3C009384F4FF1375F57FB3F43401938F0B0098
:100D4C0093D9F901630205109307F07F6302F5163E
:100D5C00B707800093943400B3E4F40093D7DB011D
:100D6C00B3E79700939F3B00130515C013070000D2
:100D7C0093162B00B3E6E6009386F6FF9305E0008E
:100D8C00334639013305AA4063E0D5169725000098
:100D9C009385C51193962600B386B60083A60600EC
:100DAC00B386B60067800600B3EA6401638E0A0658
:100DBC006380040413850400EF10502C930755FF37
:100DCC001307C001634EF702930AD001130485FF89
:100DDC00B38AFA40B3948400B35A5B01B3EA9A0025
:100DEC0033148B00130AD0C0330AAA406FF09FF360
:100DFC0013050B00EF109028130505026FF01FFC74
:100E0C00930485FDB31A9B00130400006FF09FFD43
:100E1C00B3EA640163820A02938A0400130AF07F26
:100E2C00130B30006FF05FF013040000130A000086
:100E3C00130B10006FF05FEF13040000130AF07F28
:100E4C00130B20006FF05FEEB3E77401638E07069F
:100E5C006380040413850400EF105022130755FF20
:100E6C009307C00163CEE7029307D001930F85FF70
:100E7C00B387E740B394F401B3D7FB00B3E7970013
:100E8C00B39FFB011306D0C03305A6406FF01FEED5
:100E9C0013850B00EF10901E130505026FF01FFC5D
:100EAC00930785FDB397FB00930F00006FF09FFD38
:100EBC00B3E7740163820702938704001305F07F84
:100ECC00130730006FF0DFEA930F000013050000EA
:100EDC00130710006FF0DFE9930F00001305F07F8C
:100EEC00130720006FF0DFE863E657016390FA36D2
:100EFC00636EF4359395FA01935614001317F401AD
:100F0C0093DA1A0033E4D5009397870013D88F0136
:100F1C003368F800935E0801B3D5DA03131E080199
:100F2C00135E0E019356040193988F00B3F4DA0309
:100F3C00938F0500B307BE0293940401B3E69600A9
:100F4C0063FEF600B3860601938FF5FF63E8060196
:100F5C0063F6F600938FE5FFB3860601B386F64081
:100F6C0033D3D6031314040113540401B3F6D6037C
:100F7C0093070300B3056E0293960601B366D40083
:100F8C0063FEB600B38606019307F3FF63E8060120
:100F9C0063F6B6009307E3FFB38606013384B640CD
:100FAC00939F0F01B7050100B3EFFF001383F5FF0B
:100FBC0093D60F01B3F76F0013DF080133F368000A
:100FCC00B3836702B3846602B307FF02B382E603FE
:100FDC00B386970093D70301B387D70063F49700C8
:100FEC00B382B20093D60701B3865600B702010054
:100FFC009382F2FFB3F5570093950501B3F35300B9
:10100C00B38575006368D40093870F006314D40410
:10101C006372B70433071701B3321701B3820201AD
:10102C00330454009387FFFF6366880063148802BF
:10103C00636217036366D400639E8600637CB7000B
:10104C00330717019387EFFFB33F1701B38F0F01DE
:10105C003304F401B305B7403304D4403337B7003D
:10106C003304E440930FF0FF63048812B352D403AB
:10107C0093D605013374D40313870200B30F5E02B9
:10108C001314040133E48600637EF4013304040179
:10109C001387F2FF636804016376F4011387E2FFA0
:1010AC00330404013304F441B356D403939505017E
:1010BC0093D505013374D403330EDE0213140401EB
:1010CC0033E4850093850600637EC4013304040178
:1010DC009385F6FF636804016376C4019385E6FF8C
:1010EC003304040113170701B365B7001397050107
:1010FC00135707013304C44113DE0501B30E670215
:10110C0033036E02330ECF03330FEF0213D70E01EE
:10111C00330F6F003307E70163766700B7060100F2
:10112C00330EDE00135307013303C301370E0100E6
:10113C00130EFEFFB376C70193960601B3FECE01E4
:10114C00B386D60163686400938F05006310640452
:10115C006380060433048800938FF5FF63640403F3
:10116C00636664006314640263F0D802139718007A
:10117C00B338170133880801938FE5FF330404015A
:10118C0093080700631464006384160193EF1F0037
:10119C009306F53F635AD01013F77F0063000702E4
:1011AC0013F7FF0093054000630AB70093854F00C7
:1011BC00B3BFF501B387F701938F05001397770041
:1011CC00635A0700370700FF1307F7FFB3F7E70071
:1011DC00930605401307E07F634AD7181397D7018E
:1011EC0093DF3F003367F70193D73700B705100043
:1011FC009385F5FFB3F7B700B70510809385F5FF1E
:10120C0093F6F67F93964601B3F7B7008320C1029D
:10121C00032481021316F601B3E7D700B3E6C70027
:10122C0083244102032901028329C101032A81017C
:10123C00832A4101032B0101832BC10013050700F5
:10124C009385060013010103678000001305F5FF69
:10125C00130700006FF05FCB1306090093870A0099
:10126C00930F040013070B00930620006300D710A4
:10127C00930630006302D70E93061000E31AD7F0E2
:10128C0093070000130700006F0040091386090044
:10129C006FF09FFDB7070800930F000013060000C6
:1012AC00130730006FF05FFC93051000B385D54039
:1012BC0013078003E346B7FC1307F0016344B7063A
:1012CC001305E5413397A700B3D6BF003395AF00A4
:1012DC003367D7003335A0003367A700B3D7B70007
:1012EC0093767700638006029376F70093054000AF
:1012FC00638AB6009306470033B7E600B387E7006E
:10130C00138706009396870063CA06069396D70147
:10131C001357370033E7E60093D7370093060000E6
:10132C006FF0DFEC130710FE3307D74013080002F1
:10133C0033D7E70093060000638605011305E543E8
:10134C00B396A70033E5F6013335A0003367A70049
:10135C00930700006FF0DFF8B707080013070000D1
:10136C009306F07F130600006FF05FE89307000010
:10137C00130700009306F07F6FF05FE79307000000
:10138C0013070000930610006FF05FE6130101FDD8
:10139C0023202103232A51013709100093DA450138
:1013AC00232E3101232C41012328610123267101B5
:1013BC001309F9FF2326110223248102232291020F
:1013CC0093FAFA7F130B0500930B0600138A0600A1
:1013DC003379B90093D9F50163880A0A9307F07F32
:1013EC006386FA10370480001319390033698900B9
:1013FC001354D5013364240193143500938A1AC015
:10140C00130B000013554A01370910001309F9FF9B
:10141C001375F57F3379490113870B00135AFA01C1
:10142C00630405109307F07F6304F516B70780007B
:10143C00131939003369F90093D7DB01B3E727019E
:10144C0013973B00130515C09306000093152B0052
:10145C00B3E5D5003385AA009385F5FF9308E0002A
:10146C0033C649011308150063E0B81617250000B0
:10147C00130585A793952500B385A50083A50500C5
:10148C00B385A500678005003364A900630E0406CC
:10149C006300090413050900EF10403E930755FF44
:1014AC001307C001634CF7021304D001930485FFAA
:1014BC003304F4403319990033548B003364240102
:1014CC00B3149B00930AD0C0B38AAA406FF05FF3A9
:1014DC00EF10C03A130505026FF05FFC130485FD95
:1014EC0033148B00930400006FF0DFFD3364A9000C
:1014FC00630404029304050013040900930AF07FAB
:10150C00130B30006FF01FF093040000930A0000DF
:10151C00130B10006FF01FEF93040000930AF07F81
:10152C00130B20006FF01FEEB3677901638E070673
:10153C006300090413050900EF104034930655FFAE
:10154C009307C00163CED7029307D001130785FF21
:10155C00B387D7403319E900B3D7FB00B3E72701B2
:10156C003397EB009306D0C03385A6406FF0DFEDC8
:10157C0013850B00EF108030130505026FF01FFC74
:10158C00930785FDB397FB00130700006FF09FFDD9
:10159C00B367790163820702930709001305F07F93
:1015AC00930630006FF09FEA13070000130500004C
:1015BC00930610006FF09FE9130700001305F07FEE
:1015CC00930620006FF09FE8B70F0100138FFFFF09
:1015DC0093D6040113530701B3F4E4013377E70105
:1015EC00B3089302B3059702B382E602338E580018
:1015FC0093D80501B388C801B38E660263F4580012
:10160C00B38EFE0113D90801B3F8E80193DF07018B
:10161C00B3F5E501B3F3E70193980801B388B8007B
:10162C00B3877602B3859302B3849F02338EF400A2
:10163C0093D40501B384C401B386F60363F6F400B6
:10164C00B7070100B386F60013DF0401B7090100E8
:10165C00330FDF009386F9FFB3F4D400B3F5D50054
:10166C0093570401939404013374D400B384B400ED
:10167C00B306870233099900338EE702B305830260
:10168C003307F3023383C50193D50601B385650097
:10169C0063F4C5013307370113D30501B709010002
:1016AC00B302E3001387F9FFB3F5E500B3F6E600E8
:1016BC003383830293950501B385D5003387770275
:1016CC0033848F02338EFF023304E40093570301FB
:1016DC00338487006374E400330E3E01B7070100C6
:1016EC009387F7FFB376F4003373F30093960601F8
:1016FC00B38E2E01B3866600B3B49E00B386E601AA
:10170C00B3879600B38EBE00B3B5BE0033835700CB
:10171C00B30FB300B3B6E601B3B79700B3E7F60067
:10172C001354040133335300B3B5BF00B3878700A0
:10173C00B365B300B387B700B387C70113D77F0175
:10174C0093979700B3E7E70013979E003367170151
:10175C003337E00093DE7E0193969F003367D70109
:10176C003367D7009396770063DA06109356170009
:10177C001377170033E7E6009396F7013367D7002A
:10178C0093D717009305F83F635EB00E93767700FE
:10179C00638006029376F70013054000638AA60067
:1017AC009306470033B7E600B387E70013870600BC
:1017BC009396770063DA0600B70600FF9386F6FF70
:1017CC00B3F7D700930508409306E07F63CEB616B7
:1017DC00935637001397D7013367D70093D7370049
:1017EC00B70610009386F6FFB3F7D70093F6F57F94
:1017FC00B70510809385F5FF93964601B3F7B700B4
:10180C008320C102032481021316F601B3E7D7002B
:10181C00B3E6C70083244102032901028329C101D5
:10182C00032A8101832A4101032B0101832BC1006F
:10183C001305070093850600130101036780000060
:10184C0013860900930704001387040093060B000A
:10185C0093052000638AB60E93053000638CB60C9A
:10186C0093051000E390B6F29307000013070000F5
:10187C006F00800813060A006FF09FFD1308050027
:10188C006FF05FF0130510003305B540930680032D
:10189C00E3CCA6FC9306F00163C4A6061308E8414A
:1018AC00B3960701B355A70033170701B3E6B6008B
:1018BC003337E00033E7E600B3D7A7009376770021
:1018CC00638006029376F70093054000638AB600A6
:1018DC009306470033B7E600B387E700138706008B
:1018EC009396870063CA06069396D7011357370061
:1018FC0033E7E60093D73700930500006FF05FEEF7
:10190C00930610FEB386B64093080002B3D6D700F8
:10191C0093050000630615011308E843B39507010E
:10192C0033E7E5003337E00033E7E60093070000C8
:10193C006FF0DFF8B7070800130700009305F07F7E
:10194C00130600006FF0DFE9930700001307000097
:10195C009305F07F6FF0DFE893070000130700009A
:10196C00930510006FF0DFE7130101FE232A9100AD
:10197C002326310193547501B709800023282101D6
:10198C00232441019389F9FF232E1100232C81007C
:10199C002322510193F4F40F138A0500B3F9A90023
:1019AC001359F501638804089307F00F6384F40A54
:1019BC0093993900B7070004B3E9F900938414F83C
:1019CC00930A000013557A01370480001304F4FFC6
:1019DC001375F50F33744401135AFA01630C05089F
:1019EC009307F00F6308F50A13143400B7070004CB
:1019FC003364F400130515F89307000093962A003E
:101A0C00B3E6F6009386F6FF1307E0003346490170
:101A1C003385A4406360D70A9715000093858550E1
:101A2C0093962600B386B60003A706003307B700CB
:101A3C0067000700638A090213850900EF00106430
:101A4C009307B5FF9304A0F8B399F900B384A440AD
:101A5C006FF01FF79304F00F930A2000E38409F64C
:101A6C00930A30006FF01FF693040000930A1000E5
:101A7C006FF05FF5630A040213050400EF001060B9
:101A8C009307B5FF3314F4009307A0F83385A740F0
:101A9C006FF09FF61305F00F93072000E30004F698
:101AAC00930730006FF09FF51305000093071000AB
:101ABC006FF0DFF41318540063F6890E1305F5FF6D
:101ACC00930600001354080133D38902B7070100B1
:101ADC009387F7FFB377F80093D6060133F78902A3
:101AEC0093050300B38867021317070133E7E60079
:101AFC00637E1701330707019305F3FF6368070142
:101B0C00637617019305E3FF33070701330717418A
:101B1C00B358870233778702B386170393170701ED
:101B2C001387080063FED700B38707011387F8FFFC
:101B3C0063E8070163F6D7001387E8FFB387070153
:101B4C0013940501B387D7403364E400B337F00036
:101B5C003364F4001307F5076350E00A93777400BD
:101B6C00638A07009377F400930640006384D700E0
:101B7C00130444009317440063DA0700B70700F816
:101B8C009387F7FF3374F400130705089307E00FEE
:101B9C001354340063D2E70C130400001307F00F46
:101BAC006F00800B9396F90193D919006FF09FF198
:101BBC00130609001384090093870A0013072000F9
:101BCC00E38CE7FC130730006382E708130710006F
:101BDC00E392E7F813040000130700006F00C0073E
:101BEC0013060A006FF09FFD370440001306000037
:101BFC00930730006FF09FFC93071000B387E7400A
:101C0C001307B001E348F7FC1305E509B357F400DB
:101C1C003314A4003334800033E4870093777400CA
:101C2C00638A07009377F400130740006384E7008E
:101C3C00130444009317540013543400E3DE07F8E4
:101C4C0013040000130710006F000001370440005C
:101C5C001307F00F13060000370580001305F5FF7E
:101C6C003374A400370580801305F5FF1377F70F45
:101C7C003374A400131777013364E4001315F601D1
:101C8C003365A4008320C101032481018324410115
:101C9C00032901018329C100032A8100832A410001
:101CAC001301010267800000130101FE232A910039
:101CBC0023282101B7048000135975012326310113
:101CCC00232251019384F4FF232E1100232C810035
:101CDC00232441011379F90F938A0500B3F4A4006E
:101CEC009359F501630A09089307F00F6306F90A83
:101CFC0093943400B7070004B3E4F400130919F803
:101D0C00130A000013D57A01370480001304F4FF82
:101D1C001375F50F3374540193DAFA01630E050849
:101D2C009307F00F630AF50A13143400B707000485
:101D3C003364F400130515F89306000093172A007A
:101D4C00B3E7D7003305A9009387F7FF1307E0002B
:101D5C0033C65901130815006360F70A1717000002
:101D6C001307072093972700B387E70083A7070083
:101D7C00B387E70067800700638A040213850400B9
:101D8C00EF00D02F9307B5FF1309A0F8B394F4001C
:101D9C003309A9406FF0DFF61309F00F130A200086
:101DAC00E38204F6130A30006FF0DFF5130900002C
:101DBC00130A10006FF01FF5630A040213050400E8
:101DCC00EF00D02B9307B5FF3314F4009307A0F862
:101DDC003385A7406FF05FF61305F00F93062000D4
:101DEC00E30E04F4930630006FF05FF5130500006A
:101DFC00930610006FF09FF4B70701001383F7FFF1
:101E0C0013D7040193560401B3F4640033746400D3
:101E1C00B3888402B30587023304D702B3869602D3
:101E2C0093D40801B386B600B384D40063F4B40031
:101E3C003304F400B3F7640093970701B3F8680018
:101E4C00B38717011397670093D404013337E0006D
:101E5C0093D7A70133848400B367F700131464008D
:101E6C003364F4009317440063DE070C935714009B
:101E7C001374140033E487001307F8076358E00C5D
:101E8C0093777400638A07009377F40093064000FD
:101E9C006384D700130444009317440063DA0700EB
:101EAC00B70700F89387F7FF3374F400130708089B
:101EBC009307E00F63CCE70E935734006F000003D9
:101ECC00138609001384040093060A00930720006C
:101EDC00638EF60C930730006382F60C93051000AA
:101EEC009307000013070000E398B6F8370480004E
:101EFC001304F4FF37058080B3F787001305F5FF53
:101F0C008320C101032481011377F70FB3F7A700D6
:101F1C00131777011315F601B3E7E700832441018A
:101F2C00032901018329C100032A8100832A41006E
:101F3C0033E5A700130101026780000013860A0035
:101F4C006FF0DFF8130805006FF01FF39307100014
:101F5C00B387E7401307B0016340F7061308E8099D
:101F6C00B357F400331404013334800033E4870096
:101F7C0093777400638A07009377F400130740008B
:101F8C006384E700130444009317540063CA0702E8
:101F9C0093573400130700006FF05FF5B70740004C
:101FAC001307F00F130600006FF05FF493070000A7
:101FBC001307F00F6FF09FF3930700006FF09FFD76
:101FCC0093070000130710006FF05FF2B707800053
:101FDC009387F7FF130101FF33F7A70093567501A1
:101FEC0013D67501B3F7B7002322910023202101EA
:101FFC0093F6F60F131837001376F60F23261100FD
:10200C00232481001307F00F9354F5011389060064
:10201C001305060093D5F501939737006314E6007A
:10202C006394070093C515003387C640639A951ACD
:10203C006356E00A63160606639C07009307F00FCD
:10204C00638CF60493070800138506006F00C01418
:10205C001307F7FF631E0702B387070113850600FA
:10206C0013975700635A0712130515001307F00F47
:10207C00630EE5323707007E93F617001307F7FF60
:10208C0093D71700B3F7E700B3E7D7006F00C01082
:10209C001306F00F639EC600930708006F004007FD
:1020AC001306F00FE38AC6FE37060004B3E7C70039
:1020BC001306B0016356E600930710006FF0DFF9CA
:1020CC00130600023306E640B3D5E700B397C7000A
:1020DC00B337F000B3E7F5006FF01FF863000708A3
:1020EC00639C0602631808001307F00F6316E60AD8
:1020FC006F0000029306F0FF6316D700B387070149
:10210C006FF01FF69306F00F1347F7FF6310D6021C
:10211C001305F00F6F0040089306F00FE30AD6FE8C
:10212C00B70600043307E0403368D8009306B001CB
:10213C0063D6E600130710006F00C001930600027F
:10214C003356E8003387E6403317E8003337E000B6
:10215C003367E600B387E7006FF09FF01385160036
:10216C001376F50F130710006342C7066394060439
:10217C00130500006302080263860722B387070178
:10218C0013975700635A0700370700FC1307F7FF34
:10219C00B3F7E7001305100013F77700630A072065
:1021AC0013F7F700930640006304D720938747008A
:1021BC006F000020E30E08F4E38007EEB70700027F
:1021CC001305F00F930400006F00801E1307F00F2F
:1021DC00630EE51C3307F800935717006FF0DFFB15
:1021EC006350E00863160604E38A07E41307F7FF5D
:1021FC0063140702B307F8401385060013975700C2
:10220C00E35C07F8370400041304F4FF33F487008D
:10221C00130905006F0080131306F00FE38EC6E65A
:10222C001306B0016350E602930710006FF09FFC99
:10223C001306F00FE382C6E637060004B3E7C700C7
:10224C006FF01FFE13060002B3D5E7003307E6401C
:10225C00B397E700B337F000B3E7F5006FF09FF9E1
:10226C0063020708639E0602631808001307F00F49
:10227C00938405006FF09FE79306F0FF6318D70077
:10228C00B3870741938405006FF05FF79306F00F57
:10229C001347F7FF6310D602938405006FF05FE7D6
:1022AC009306F00FE30AD6FEB70600043307E040AE
:1022BC003368D8009306B00163D6E600130710000C
:1022CC006F00C001930600023356E8003387E640E6
:1022DC003317E8003337E0003367E600B387E74095
:1022EC006FF05FFA138716001377F70F13061000C1
:1022FC006344E604639C06026318080063980712A3
:10230C00130500006FF01FEC638607123307F840CB
:10231C0093165700B387074163CA0610930707004B
:10232C0063100706930700006FF09FFDE31608E8A3
:10233C00E39407F66FF09FE83304F840131754004A
:10234C006354070433840741938405001305040088
:10235C00EF00C0521305B5FF3314A400634A2503E4
:10236C00330525411305150013070002B357A400CC
:10237C003305A7403314A40033348000B3E787003F
:10238C00130500006FF05FE1E30E04F86FF01FFC23
:10239C00B70700FC9387F7FF3305A940B377F40028
:1023AC006FF09FDF930708006FF01FDF93070000AB
:1023BC0013975700635E0700130515001307F00F02
:1023CC00630EE506370700FC1307F7FFB3F7E700CA
:1023DC001307F00F93D737006318E50063860700E7
:1023EC00B707400093040000370780001307F7FF7E
:1023FC001375F50FB3F7E7001317750137058080D8
:10240C008320C100032481001305F5FF33F5A700D9
:10241C009394F4013365E5003365950003290100BD
:10242C00832441001301010167800000938405009F
:10243C006FF01FF5930708006FF09FF493070000EF
:10244C006FF01FF937068000135775019307F6FFDD
:10245C001377F70F9305E007B3F7A7009356F50131
:10246C0063F6E5049305D00963FAE50037050080AF
:10247C001345F5FF3385A6006780000033E5C700E0
:10248C009307500963DCE7001307A7F63315E50043
:10249C00638006023305A040678000009307600943
:1024AC003387E7403355E5006FF09FFE13050000BE
:1024BC0067800000130101FF2326110023248100F3
:1024CC002322910063020510130405009354F501B7
:1024DC00635405003304A04013050400EF00003AD8
:1024EC009307E009B387A740130760096340F70619
:1024FC00130780006356A700130585FF3314A4004F
:10250C00370580001305F5FF93F7F70F3374A4001C
:10251C0013957701B70780809387F7FF3374F40026
:10252C00B70700803364A40093C7F7FF1395F40139
:10253C003374F4003365A4008320C10003248100AC
:10254C0083244100130101016780000013079009E7
:10255C006350F702130750003307A7409306B501E9
:10256C003357E4003314D4003334800033648700D1
:10257C00130750006356A7001307B5FF3314E4008C
:10258C00370700FC1307F7FF937674003377E400EA
:10259C00638A06001374F400930640006304D400AD
:1025AC00130747009316570063DC0600B70700FCBF
:1025BC009387F7FF3377F7009307F009B387A740AA
:1025CC00135437006FF0DFF313040000930700007F
:1025DC00930400006FF0DFF293577501130101FFB4
:1025EC0093F7F70F2324810013871700370480001B
:1025FC00232291001304F4FF232611001377F70F05
:10260C00930610003374A4009354F50163D2E606CC
:10261C0013850738935734001314D401370710006F
:10262C001307F7FFB3F7E700370710801307F7FF1F
:10263C001375F57F13154501B3F7E70037070080D5
:10264C00B3E7A7001347F7FF1395F401B3F7E700BF
:10265C0033E7A7008320C100130504000324810085
:10266C0083244100930507001301010167800000DA
:10267C00639407046302040613050400EF000020B2
:10268C009307A00063C2A7029307B000B387A740CB
:10269C0013075501B357F4003314E40013079038B3
:1026AC003305A7406FF09FF7930755FFB317F4005E
:1026BC00130400006FF09FFE93070000630A0400F0
:1026CC0093573400370708001314D401B3E7E7001D
:1026DC001305F07F6FF09FF49307000013050000C3
:1026EC006FF0DFF3370610001306F6FF3376B600F3
:1026FC0013D845019357D5011378F87F131636007C
:10270C0033E6C7009307180093F7F77F9306100082
:10271C0093D5F5011317350063D6F60A930608C84E
:10272C009307E00F63C2D70C6340D008930790FE69
:10273C0063C4F612B70780001305E0013366F60098
:10274C003305D5409307F00163C8A702130828C8C6
:10275C00B3170701B337F000331606013355A70042
:10276C00B3E7C700B367F5009306000013F77700D3
:10277C00630007086F00C00E9307E0FFB386D740D5
:10278C0093070002B356D600930800006306F500C9
:10279C00130828CAB3180601B3E7E800B337F000F2
:1027AC00B3E7F6006FF05FFC131565003335A0003E
:1027BC00131636009357D7013366C500B367F6007E
:1027CC006FF0DFFAB367E60063160800B337F0006A
:1027DC006FF09FF99306F00F638C07001316360009
:1027EC00B70700026FF09FFD930700009306F00FF0
:1027FC0013975700635E0700938616001307F00FBC
:10280C00638AE606370700FC1307F7FFB3F7E70008
:10281C001307F00F93D737006398E6006386070021
:10282C00B707400093050000370580001305F5FF3E
:10283C00B3F7A700370580801305F5FF93F6F60F65
:10284C0093967601B3F7A7009395F501B3E7D700FC
:10285C0033E5B70067800000930710009306000073
:10286C0013F7F70013064000E304C7F893874700FB
:10287C006FF01FF8930700006FF09FF9B707010086
:10288C00637AF5029307F00FB3B7A700939737005D
:10289C00130700023307F740B357F5001705000084
:1028AC001305C56FB307F50003C507003305A74033
:1028BC00678000003707000193070001E36AE5FC1D
:0828CC00930780016FF0DFFCAF
:1028D400411106C6EFD05F94B240B70710F023A0B1
:0828E40007F201454101828069
:1028EC004448525953544F4E452050524F47524131
:1028FC004D2C20534F4D4520535452494E47000008
:10290C004468727973746F6E652042656E63686D8E
:10291C0061726B2C2056657273696F6E20322E318A
:10292C0020284C616E67756167653A204329000069
:10293C0050726F6772616D20636F6D70696C656446
:10294C0020776974682027726567697374657227CC
:10295C0020617474726962757465000050726F67DF
:10296C0072616D20636F6D70696C6564207769743A
:10297C00686F757420277265676973746572272098
:10298C00617474726962757465000000506C6561E5
:10299C007365206769766520746865206E756D6255
:1029AC006572206F662072756E73207468726F7515
:1029BC006768207468652062656E63686D61726B10
:1029CC003A200000457865637574696F6E207374E6
:1029DC00617274732C2025642072756E7320746878
:1029EC00726F756768204468727973746F6E650ACC
:1029FC0000000000457865637574696F6E20656E24
:102A0C006473000046696E616C2076616C75657349
:102A1C00206F6620746865207661726961626C65EE
:102A2C0073207573656420696E2074686520626517
:102A3C006E63686D61726B3A00000000496E745FE2
:102A4C00476C6F623A20202020202020202020205C
:102A5C002025640A000000002020202020202020B7
:102A6C0073686F756C642062653A20202025640AB7
:102A7C0000000000426F6F6C5F476C6F623A202061
:102A8C0020202020202020202025640A0000000087
:102A9C0043685F315F476C6F623A20202020202012
:102AAC00202020202025630A000000002020202068
:102ABC002020202073686F756C642062653A20209A
:102ACC002025630A0000000043685F325F476C6F8B
:102ADC00623A202020202020202020202025630A5C
:102AEC00000000004172725F315F476C6F625B38AF
:102AFC005D3A2020202020202025640A00000000C0
:102B0C004172725F325F476C6F625B385D5B375D41
:102B1C003A2020202025640A0000000020202020DC
:102B2C002020202073686F756C642062653A202029
:102B3C00204E756D6265725F4F665F52756E7320C5
:102B4C002B203130000000005074725F476C6F62B4
:102B5C002D3E000020205074725F436F6D703A2040
:102B6C0020202020202020202025640A00000000A6
:102B7C00202020202020202073686F756C64206238
:102B8C00653A20202028696D706C656D656E7461E6
:102B9C0074696F6E2D646570656E64656E74290062
:102BAC00202044697363723A2020202020202020AA
:102BBC00202020202025640A000000002020456EE3
:102BCC00756D5F436F6D703A2020202020202020EF
:102BDC002025640A000000002020496E745F436FBA
:102BEC006D703A2020202020202020202025640AEF
:102BFC000000000020205374725F436F6D703A2008
:102C0C0020202020202020202025730A00000000F6
:102C1C00202020202020202073686F756C64206297
:102C2C00653A2020204448525953544F4E45205069
:102C3C00524F4752414D2C20534F4D452053545227
:102C4C00494E47004E6578745F5074725F476C6FE5
:102C5C00622D3E00202020202020202073686F75DC
:102C6C006C642062653A20202028696D706C656D5B
:102C7C00656E746174696F6E2D646570656E6465E4
:102C8C006E74292C2073616D652061732061626FF5
:102C9C0076650000496E745F315F4C6F633A20209B
:102CAC0020202020202020202025640A0000000065
:102CBC00496E745F325F4C6F633A202020202020D5
:102CCC00202020202025640A00000000496E745F3B
:102CDC00335F4C6F633A20202020202020202020BE
:102CEC002025640A00000000456E756D5F4C6F6313
:102CFC003A20202020202020202020202025640A7B
:102D0C00000000005374725F315F4C6F633A2020F7
:102D1C0020202020202020202025730A00000000E5
:102D2C00202020202020202073686F756C64206286
:102D3C00653A2020204448525953544F4E45205058
:102D4C00524F4752414D2C2031275354205354524B
:102D5C00494E47005374725F325F4C6F633A2020C8
:102D6C0020202020202020202025730A0000000095
:102D7C00202020202020202073686F756C64206236
:102D8C00653A2020204448525953544F4E45205008
:102D9C00524F4752414D2C2032274E44205354520F
:102DAC00494E47004D656173757265642074696D99
:102DBC006520746F6F20736D616C6C20746F206F65
:102DCC00627461696E206D65616E696E6766756CA3
:102DDC0020726573756C747300000000506C656133
:102DEC00736520696E637265617365206E756D62C3
:102DFC006572206F662072756E730000436C6F6392
:102E0C006B206379636C65733D2564200A000000B8
:102E1C00444D49505320706572204D687A3A2020F9
:102E2C002020202020202020202020202020202096
:102E3C002020202020202020202020200000000006
:102E4C0025642E00256400004448525953544F4EBB
:102E5C00452050524F4752414D2C2031275354207E
:102E6C00535452494E4700004448525953544F4E04
:102E7C00452050524F4752414D2C2032274E442072
:102E8C00535452494E4700004448525953544F4EE4
:102E9C00452050524F4752414D2C2033275244204D
:102EAC00535452494E470000C4E4FFFFD8E3FFFFE0
:102EBC00E4E3FFFFD8E3FFFFB0E4FFFFD8E3FFFF3D
:102ECC00E4E3FFFFC4E4FFFFC4E4FFFFB0E4FFFF53
:102EDC00E4E3FFFFB0E3FFFFB0E3FFFFB0E3FFFF6E
:102EEC00ECE3FFFF6CE9FFFF6CE9FFFF90E9FFFFEC
:102EFC0060E9FFFF60E9FFFF50EAFFFF90E9FFFF89
:102F0C0060E9FFFF50EAFFFF60E9FFFF90E9FFFF78
:102F1C005CE9FFFF5CE9FFFF5CE9FFFF50EAFFFFA4
:102F2C0078ECFFFFB4ECFFFFC0ECFFFFB4ECFFFF4D
:102F3C002CEDFFFFB4ECFFFFC0ECFFFF78ECFFFFC4
:102F4C0078ECFFFF2CEDFFFFC0ECFFFF90ECFFFFD8
:102F5C0090ECFFFF90ECFFFFC8ECFFFF70EFFFFF62
:102F6C0070EFFFFFE0EFFFFF68EFFFFF68EFFFFF81
:102F7C0040F0FFFFE0EFFFFF68EFFFFF40F0FFFFC7
:102F8C0068EFFFFFE0EFFFFF64EFFFFF64EFFFFF71
:102F9C0064EFFFFF40F0FFFF000102020303030395
:102FAC0004040404040404040505050505050505CD
:102FBC0005050505050505050606060606060606AD
:102FCC000606060606060606060606060606060695
:102FDC00060606060606060607070707070707077D
:102FEC000707070707070707070707070707070765
:102FFC000707070707070707070707070707070755
:10300C000707070707070707070707070707070744
:10301C00070707070707070708080808080808082C
:10302C000808080808080808080808080808080814
:10303C000808080808080808080808080808080804
:10304C0008080808080808080808080808080808F4
:10305C0008080808080808080808080808080808E4
:10306C0008080808080808080808080808080808D4
:10307C0008080808080808080808080808080808C4
:10308C0008080808080808080808080808080808B4
:08309C000808080808080808EC
:1030A8000000000080842E41000000205FA0124232
:0C30B800F90295503353DE470000C84277
:040000058000000077
:00000001FF
